:1000000012C0189518951895189518951895189563
:100010001895189518951895189518951895189578
:100020001895189518958FED8DBFC0ECE0EC4E2E0D
:10003000DD275D2EEEE7F0E0A0E6B0E088278D93A7
:100040003197E9F7662481EF87BB8FE788BB8FE79D
:1000500081BB8FE782BBC798C49A0027A6E38C9127
:1000600083FB0EF401E041E0041781E009F080E039
:100070008F930027A6E38C9182FB0EF401E040E011
:10008000041781E009F080E09F9189238F93002776
:10009000A6E38C9181FB0EF401E041E0041781E0BE
:1000A00009F080E09F918923882309F485C0C698D0
:1000B000C79A0027A6E38C9183FB0EF401E041E090
:1000C000041781E009F080E08F930027A6E38C916C
:1000D00082FB0EF401E040E0041781E009F080E0CB
:1000E0009F9189238F930027A6E38C9181FB0EF4C7
:1000F00001E041E0041781E009F080E09F9189234D
:10010000882309F459C0C598C69A0027A6E38C91A4
:1001100083FB0EF401E041E0041781E009F080E088
:100120008F930027A6E38C9182FB0EF401E041E05F
:10013000041781E009F080E09F9189238F930027C5
:10014000A6E38C9181FB0EF401E041E0041781E00D
:1001500009F080E09F918923882309F42DC0C49879
:10016000C59A0027A6E38C9183FB0EF401E040E0E2
:10017000041781E009F080E08F930027A6E38C91BB
:1001800082FB0EF401E041E0041781E009F080E019
:100190009F9189238F930027A6E38C9181FB0EF416
:1001A00001E040E0041781E009F080E09F9189239D
:1001B000882309F401C065D29FD29ED29DD281E0EE
:1001C0008093610081D146D0009160000C3008F02E
:1001D0003EC0009160000A3008F01AC00091610032
:1001E000053008F00DC080916000A1E6AD90A1E659
:1001F000AA0D8C93809166008F778093660004C06F
:1002000063D185E080936100A1E68C918F5F8C9330
:10021000009160000A3009F011C00027A6E68C9119
:1002200087FB0EF401E041E0041709F006C06DD22F
:1002300081E08093610048D101C089D100916000C4
:100240000B3009F004C081E0809361003DD1BBCF49
:10025000F894FFCF8FEF80936000C798C49A00276F
:10026000A6E38C9183FB0EF401E040E0041709F053
:100270000FC081E0809360003FD20027A6E38C91FD
:1002800083FB0EF401E040E0041709F001C0F5CF54
:100290000027A6E38C9182FB0EF401E040E00417F6
:1002A00009F00FC082E08093600026D20027A6E309
:1002B0008C9182FB0EF401E040E0041709F001C0CC
:1002C000F5CF0027A6E38C9181FB0EF401E040E01E
:1002D000041709F00FC083E0809360000DD200275F
:1002E000A6E38C9181FB0EF401E040E0041709F0D5
:1002F00001C0F5CFC698C79A0027A6E38C9183FB6F
:100300000EF401E040E0041709F00FC084E0809390
:100310006000F2D10027A6E38C9183FB0EF401E08C
:1003200040E0041709F001C0F5CF0027A6E38C9147
:1003300082FB0EF401E040E0041709F00FC085E0F5
:1003400080936000D9D10027A6E38C9182FB0EF444
:1003500001E040E0041709F001C0F5CF0027A6E353
:100360008C9181FB0EF401E040E0041709F00FC00E
:1003700086E080936000C0D10027A6E38C9181FBCA
:100380000EF401E040E0041709F001C0F5CFC59874
:10039000C69A0027A6E38C9183FB0EF401E040E0AF
:1003A000041709F00FC087E080936000A5D10027F3
:1003B000A6E38C9183FB0EF401E040E0041709F002
:1003C00001C0F5CF0027A6E38C9182FB0EF401E07B
:1003D00040E0041709F00FC088E0809360008CD1E2
:1003E0000027A6E38C9182FB0EF401E040E00417A5
:1003F00009F001C0F5CF0027A6E38C9181FB0EF434
:1004000001E040E0041709F00FC089E0809360002C
:1004100073D10027A6E38C9181FB0EF401E040E04C
:10042000041709F001C0F5CFC498C59A0027A6E3C8
:100430008C9183FB0EF401E040E0041709F00EC03C
:100440008AE0809360000027A6E38C9183FB0EF482
:1004500001E040E0041709F001C0F5CF0027A6E352
:100460008C9182FB0EF401E040E0041709F00FC00C
:1004700080E08093600040D10027A6E38C9182FB4E
:100480000EF401E040E0041709F001C0F5CF0027A9
:10049000A6E38C9181FB0EF401E040E0041709F023
:1004A0000FC08BE08093600027D10027A6E38C91DA
:1004B00081FB0EF401E040E0041709F001C0F5CF24
:1004C0008AE090E049D1089584E68093620084E652
:1004D0008093630084E68093640084E680936500E3
:1004E0008091660080688093660008958091660020
:1004F00080648093660081E08093680000916800CA
:10050000043010F009F022C00091680040916900A9
:10051000040FAAE60C93AAE6EC91FF27A7E691E068
:1005200043D1A8E6AD90A1E6AA0D4C9100916700D9
:10053000041709F405C0809166008F7B80936600E4
:10054000A8E68C918F5F8C9308F4D8CF089580E053
:1005500080936900CBDFA6E68C9186FBA6E68C91A2
:1005600085F98C9384E080936900C0DFA6E68C91C6
:1005700086FBA6E68C9184F98C9388E080936900D1
:10058000B5DFA6E68C9186FBA6E68C9183F98C9369
:100590008CE080936900AADFA6E68C9186FBA6E634
:1005A0008C9182F98C930027A6E68C9185FB0EF442
:1005B00001E041E0041781E009F080E08F9300271B
:1005C000A6E68C9184FB0EF401E041E0041781E083
:1005D00009F080E09F91892B8F930027A6E68C91EC
:1005E00083FB0EF401E041E0041781E009F080E0B4
:1005F0009F91892B8F930027A6E68C9182FB0EF4A6
:1006000001E041E0041781E009F080E09F91892B2F
:10061000882309F434C070D06FD06ED00027A6E6CE
:100620008C9185FB0EF401E041E0041709F001C054
:1006300072D00027A6E68C9184FB0EF401E041E025
:10064000041709F001C06DD00027A6E68C9183FB4A
:100650000EF401E041E0041709F001C068D0002762
:10066000A6E68C9182FB0EF401E041E0041709F04C
:1006700001C063D081E08093610026DF01C045D0D6
:10068000089543D084EF91E067D03FD084EF91E0AC
:1006900063D03BD081E080936100DCDD009160009D
:1006A0000C3008F027C000916000093010F009F00C
:1006B00001C003C084E680936000A1E6EC91FF27AF
:1006C000A0E691E07BE75FD00091610044E073D049
:1006D000A8E68C9300916800003009F001C015D0A5
:1006E000A1E68C918F5F8C9300916100013109F03C
:1006F00001C001C0D2CF0895C09884E690E02CD00C
:10070000C09A84E690E028D00895C09888EE93E0DF
:1007100023D0C09A0895929880E293E01DD0929AD7
:100720000895939880E293E017D0939A089594984F
:1007300080E293E011D0949A0895959880E293E036
:100740000BD0959A08953197F1F70895689462F85F
:100750000895E89462F80895EF93FF93EE27E82B4D
:10076000E92B31F0E8EEF3E03197F1F70197D1F79B
:10077000FF91EF910895E199FECFEEBB3196089578
:1007800091E001C092E07B3751F47FB7F894F3DF3A
:100790008D918DBBE29AE19A9A95C9F77FBF772731
:1007A000089591E001C092E0E6DFE09A8DB38D9369
:1007B0009A95D1F70895FF93881BF9E0001FFA95E9
:1007C00011F4FF910895881F841B18F4840F8894F6
:0607D000F5CF0894F3CF01
:00000001FF
